:100000000C9400010C941D010C941D010C941D0115
:100010000C941D010C941D010C941D010C941D01E8
:100020000C941D010C941D010C941D010C941D01D8
:100030000C941D010C941D010C941D010C941D01C8
:100040000C941D010C941D010C941D010C941D01B8
:100050000C941D01BB09B10996098709A1097E0904
:1000600071097A096D09030DE40CCD0C4A0A4A0A9C
:100070004A0A4A0A4A0A4A0A4A0A4A0A4A0A4A0AE0
:100080004A0A4A0A4A0A4A0A4A0A4A0A4A0A4A0AD0
:100090004A0A4A0A4A0A4A0A4A0A4A0A4A0A4A0AC0
:1000A0004A0A4A0A4A0A4A0A4A0A4A0A4A0A4A0AB0
:1000B0004A0A4A0A4A0AC40C5F0D170D950C760CC1
:1000C000CD0DAE0DE50DB20C6F0D680D820D820DDC
:1000D0007A0B120C070CFB0BF10BE10BD40B8B0B07
:1000E0004A0A4A0A4A0A4A0A4A0A4A0A4A0A4A0A70
:1000F0004A0A4A0A4A0A4A0A4A0A4A0A4A0A4A0A60
:100100004A0A4A0A4A0A4A0A800B6B0C5C0C220C07
:10011000180C4A0A4A0A4A0A700B660B4A0A4A0A2B
:100120004A0A4A0A4A0A4A0A4A0A4A0A4A0A4A0A2F
:100130004A0A4A0A4A0A4A0A4A0A4A0A4A0A4A0A1F
:100140004A0A4A0A4A0A4A0A4A0A4A0A4A0A4A0A0F
:100150004A0A4A0A4A0A5B0B3D0B2A0BF90A4A0A69
:100160004A0A4A0A4A0A4A0A4A0A4A0A4A0A4A0AEF
:100170004A0A4A0A4A0A4A0A4A0A4A0A4A0A4A0ADF
:100180004A0A4A0A4A0A4A0A4A0A4A0A4A0A4A0ACF
:100190004A0A4A0A4A0A4A0A4A0A4A0A4A0A4A0ABF
:1001A0004A0A4A0A4A0ACD0AAD0A4A0A4A0A4A0AC9
:1001B0004A0A4A0A4A0A4A0A4A0A4A0A4A0A4A0A9F
:1001C0004A0A4A0A4A0A4A0A4A0A4A0A4A0A4A0A8F
:1001D0004A0A4A0A4A0A4A0A4A0A4A0A4A0A4A0A7F
:1001E0004A0A4A0A4A0A4A0A4A0A4A0A4A0A4A0A6F
:1001F0004A0A4A0A4A0A910A820A6579312E30006F
:1002000011241FBECFE5D8E0DEBFCDBF10E0A0E6D1
:10021000B0E0E2E6FDE102C005900D92A636B1071E
:10022000D9F727E0A6E6B0E001C01D92AA37B207D1
:10023000E1F70E94ED090C94AF0E0C94000091ECD4
:1002400096B94431510570F04832510508F049C063
:1002500092EC9093740708C0403491E0590708F479
:100260004FC096EC9093740792E09EBD806687B96C
:1002700041505109AF9A349BFECF329A10927907C0
:10028000109278076115710549F11DBC1CBC809165
:10029000740786B9349BFECF8091760790917707DB
:1002A0009C012F5F3F4F309377072093760725B14E
:1002B000FC01E759FF4F2083329A8CB590E08417F8
:1002C0009507D8F3809178079091790701969093DC
:1002D00079078093780786179707B8F216B8AF9812
:1002E00008954035510540F0403A510508F0B4CF2B
:1002F00094EC90937407B8CF93EC90937407B4CFB9
:1003000095EC90937407B0CF0F931F93CF93DF9327
:10031000282F217030E0220F331F522F5160E82F19
:10032000E270E160847090E095958795382F316098
:10033000425082E08EBDAF9A1092790710927807F2
:100340006115710509F486C0A3E020E194E1FCE1A8
:100350001CBCA8BB22BB92BB22BB92BB38BB22BB3E
:1003600092BBE8BB22BB92BB58BB22BB92BB92BBE9
:1003700022BB22BB92BB22BB92BB22BB92BB86B3E9
:1003800081708093730722BB92BB86B3B0917307D1
:10039000BB0F81708B2B8093730722BB92BB86B3FC
:1003A000B0917307BB0F81708B2B8093730722BBB7
:1003B00092BB86B3B0917307BB0F81708B2B809378
:1003C000730722BB92BB86B3B0917307BB0F8170DA
:1003D0008B2B8093730722BB92BB86B3B0917307BC
:1003E000BB0F81708B2B8093730722BB92BB86B3AC
:1003F000B0917307BB0F81708B2B8093730722BB67
:1004000092BB86B3B0917307BB0F81708B2B809327
:100410007307F2BB8CB58417E8F3C0917607D091CF
:1004200077078E010F5F1F4F1093770700937607B2
:10043000C759DF4F809173078883C0917807D091A7
:1004400079072196D0937907C0937807C617D70705
:1004500008F47ECFAF98DF91CF911F910F9108954F
:100460000F931F93CF93DF93282F217030E0220F3B
:10047000331F522F5160E82FE270E160847090E0EA
:1004800095958795382F3160425082E08EBDAF9AA6
:1004900010927907109278076115710509F489C0E7
:1004A000A3E020E194E1FCE11CBCA8BB22BB92BB11
:1004B00022BB92BB38BB22BB92BBE8BB22BB92BB28
:1004C00058BB22BB92BB92BB22BB22BB92BB22BBBE
:1004D00092BB22BB92BB86B381708093730722BB11
:1004E00092BB86B3B0917307BB0F81708B2B809347
:1004F000730722BB92BB86B3B0917307BB0F8170A9
:100500008B2B8093730722BB92BB86B3B09173078A
:10051000BB0F81708B2B8093730722BB92BB86B37A
:10052000B0917307BB0F81708B2B8093730722BB35
:1005300092BB86B3B0917307BB0F81708B2B8093F6
:10054000730722BB92BB86B3B0917307BB0F817058
:100550008B2B8093730722BB92BB86B3B09173073A
:10056000BB0F81708B2B80937307F2BB8CB5841704
:10057000E8F3000000000000C0917607D0917707F3
:100580008E010F5F1F4F1093770700937607C759AF
:10059000DF4F809173078883C0917807D0917907E6
:1005A0002196D0937907C0937807C617D70708F428
:1005B0007BCFAF98DF91CF911F910F910895CF938B
:1005C000DF93AC0182E08EBD660F6250AF9A10924D
:1005D0007907109278074115510509F4F5C073E0C9
:1005E00020E194E1F1E0ECE11CBC78BB22BB92BBC2
:1005F00022BB92BBF8BB22BB92BB22BB92BB22BBED
:1006000092BB92BB22BB22BB92BB22BB92BB22BB42
:1006100092BB86B381708093730722BB92BB86B373
:1006200030917307330F8170832B8093730722BB44
:1006300092BB86B330917307330F8170832B809305
:10064000730722BB92BB86B330917307330F81705F
:10065000832B8093730722BB92BB86B330917307C1
:10066000330F8170832B8093730722BB92BB86B3B9
:1006700030917307330F8170832B8093730722BBF4
:1006800092BB86B330917307330F8170832B8093B5
:10069000730722BB92BB86B330917307330F81700F
:1006A000832B80937307E2BBA0917607B091770705
:1006B000ED012196D0937707C0937607A759BF4FD6
:1006C000809173078C9378BB22BB92BB22BB92BBF9
:1006D000F8BB22BB92BB22BB92BB78BB22BB92BBB6
:1006E00092BB22BB22BB92BB22BB92BB22BB92BB62
:1006F00086B381708093730722BB92BB86B330911F
:100700007307330F8170832B8093730722BB92BBD7
:1007100086B330917307330F8170832B80937307F7
:1007200022BB92BB86B330917307330F8170832B4A
:100730008093730722BB92BB86B330917307330F4C
:100740008170832B8093730722BB92BB36B3809159
:100750007307880F3170382B3093730722BB92BB1D
:1007600036B380917307880F3170382B309373073D
:1007700022BB92BB36B380917307880F3170382B40
:1007800030937307E2BB3CB53617E8F3A0917607C8
:10079000B0917707ED012196D0937707C093760744
:1007A000A759BF4F809173078C9300000000A09160
:1007B0007807B09179071196B0937907A0937807DD
:1007C000A417B50708F410CFAF98DF91CF91089523
:1007D000EF92FF920F931F93CF93DF93282F2170F7
:1007E00030E0220F331F922F9160F92EA82FA270B4
:1007F000A160847090E095958795E82FE160EE2EDA
:100800004250510982E08EBDAF9A10927907109242
:1008100078076115710509F4DEC0C3E080E194E159
:10082000BCE11DBC1CBCC8BB82BB82BB92BB92BBE3
:1008300082BB82BB92BBE8BA82BB82BB92BBA8BB25
:1008400082BB82BB92BBF8BA82BB82BB92BB92BB1B
:1008500092BB92BB92BB92BB82BB82BB92BB92BB50
:1008600092BB92BB92BB92BB82BB82BB92BB92BB40
:1008700082BB82BB92BB26B321702093730782BBDD
:1008800082BB92BB26B330917307330F2170232BA9
:100890002093730782BB82BB92BB26B33091730750
:1008A000330F2170232B2093730782BB82BB92BB33
:1008B00026B330917307330F2170232B20937307D6
:1008C00082BB82BB92BB26B330917307330F21707A
:1008D000232B2093730782BB82BB92BB26B330913C
:1008E0007307330F2170232B2093730782BB82BBC6
:1008F00092BB26B330917307330F2170232B2093C3
:10090000730782BB82BB92BB26B330917307330F50
:100910002170232B2093730782BB82BB92BB26B32B
:1009200021702093740782BB82BB92BB26B33091A7
:100930007407330F2170232B2093740782BB82BB73
:1009400092BB26B330917407330F2170232B209371
:10095000740782BB82BB92BB26B330917407330FFE
:100960002170232B20937407B2BB209164002230A6
:10097000D0F1009176071091770798012F5F3F4FD4
:1009800007591F4FD0917407D295D07FF801D083BB
:1009900089010F5F1F4F1093770700937607275940
:1009A0003F4FD0917307F901D0832CB53DB5241783
:1009B0003507D8F30000000000002091780730913F
:1009C00079072F5F3F4F30937907209378072617D9
:1009D000370708F426CFAF98DF91CF911F910F9181
:1009E000FF90EF9008952091760730917707D0CF50
:1009F000FF920F931F93CF93DF93FC0161507048D8
:100A0000660F771F82E08EBDAF9A10927907109221
:100A10007807309709F4A4C1B3E090E124E1A1E0A4
:100A20008CE1F82E1DBC1CBCB8BB92BB92BB22BB98
:100A300022BB92BB92BB22BBA8BB92BB92BB22BB88
:100A4000A8BB92BB92BB22BBA8BB92BB92BB22BBF2
:100A500022BB22BB22BB22BB22BB92BB92BB22BBCE
:100A600022BB22BB22BB22BB22BB92BB92BB22BBBE
:100A700022BB92BB92BB22BB86B38170809373076B
:100A800092BB92BB22BB86B330917307330F817048
:100A9000832B8093730792BB92BB22BB86B33091AA
:100AA0007307330F8170832B8093730792BB92BBC4
:100AB00022BB86B330917307330F8170832B8093F1
:100AC000730792BB92BB22BB86B330917307330F7F
:100AD0008170832B8093730792BB92BB22BB86B33A
:100AE00030917307330F8170832B8093730792BB10
:100AF00092BB22BB86B330917307330F8170832B77
:100B00008093730792BB92BB22BB86B3309173076D
:100B1000330F8170832B8093730792BB92BB22BBF0
:100B200086B381708093740792BB92BB22BB86B35D
:100B300030917407330F8170832B8093740792BBBD
:100B400092BB22BB86B330917407330F8170832B25
:100B50008093740792BB92BB22BB86B3309174071B
:100B6000330F8170832B80937407F2BA80916400F5
:100B7000823008F4FCC00091760710917707A80135
:100B80004F5F5F4F07591F4F809174078295807F99
:100B9000E80188838A010F5F1F4F10937707009346
:100BA000760747595F4F80917307EA018883B8BB86
:100BB00092BB92BB22BB22BB92BB92BB22BBA8BB07
:100BC00092BB92BB22BBA8BB92BB92BB22BBB8BB61
:100BD00092BB92BB22BB22BB22BB22BB22BB22BB4D
:100BE00092BB92BB22BB22BB22BB22BB22BB22BB3D
:100BF00092BB92BB22BB22BB92BB92BB22BB86B3F1
:100C000081708093730792BB92BB22BB86B33091F5
:100C10007307330F8170832B8093730792BB92BB52
:100C200022BB86B330917307330F8170832B80937F
:100C3000730792BB92BB22BB86B330917307330F0D
:100C40008170832B8093730792BB92BB22BB86B3C8
:100C500030917307330F8170832B8093730792BB9E
:100C600092BB22BB86B330917307330F8170832B05
:100C70008093730792BB92BB22BB86B330917307FC
:100C8000330F8170832B8093730792BB92BB22BB7F
:100C900086B330917307330F8170832B8093730772
:100CA00092BB92BB22BB86B381708093740792BBC8
:100CB00092BB22BB36B380917407880F3170382BFA
:100CC0003093740792BB92BB22BB36B380917407FA
:100CD000880F3170382B3093740792BB92BB22BBC4
:100CE00036B380917407880F3170382B30937407B6
:100CF000F2BA80916400823008F43EC00091760719
:100D000010917707A8014F5F5F4F07591F4F8091E0
:100D100074078295807FE80188838A010F5F1F4FE7
:100D2000109377070093760747595F4F80917307B9
:100D3000EA0188834CB55DB546175707D8F3000024
:100D40000000000040917807509179074F5F5F4F96
:100D500050937907409378074E175F0708F462CEE7
:100D6000AF98DF91CF911F910F91FF90089540911F
:100D70007607509177070ECF40917607509177070D
:100D8000CCCF33E038BB90E192BB92BB24E122BBD5
:100D900022BB92BB92BB22BB82FFB7C038BB90E1A3
:100DA00092BB92BB94E192BB81FFACC093E098BB35
:100DB00090E192BB92BB94E192BB80FFA0C083E024
:100DC00088BB80E182BB82BB94E192BB82BB82E0A4
:100DD0008EBD1DBC1CBC909163008CB58917E8F3D7
:100DE00094E192BB92BB80E182BB82BB92BB92BB7F
:100DF00082BB82BB92BB26B321702093730782BB58
:100E000082BB92BB26B330917307330F2170232B23
:100E10002093730782BB82BB92BB26B330917307CA
:100E2000330F2170232B2093730782BB82BB92BBAD
:100E300026B330917307330F2170232B2093730750
:100E400082BB82BB92BB26B321702093740782BB06
:100E500082BB92BB26B330917407330F2170232BD2
:100E60002093740782BB82BB92BB26B33091740778
:100E7000330F2170232B2093740782BB82BB92BB5C
:100E800026B330917407330F2170232B20937407FE
:100E900082BB82BB92BB26B330917407330F2170A3
:100EA000232B2093740782BB82BB92BB26B3309165
:100EB0007407330F2170232B2093740782BB82BBEE
:100EC00092BB26B330917407330F2170232B2093EC
:100ED000740782BB82BB92BB86B390917407990F53
:100EE0008170892B809374078CE182BB809173079A
:100EF00090E0982F882720917407822B089581E035
:100F000088BB5FCF91E098BB53CF91E098BB47CFB0
:100F1000282F217030E0220F331F322F3160482FED
:100F200042704160847090E095958795816093E070
:100F300098BB20E122BB94E192BB22BB92BB88BB51
:100F400022BB92BB48BB22BB92BB38BB22BB92BB2D
:100F500092BB22BB22BB92BB22BB92BB22BB92BBE9
:100F600086B381708093730722BB92BB86B33091A6
:100F70007307330F8170832B8093730722BB92BB5F
:100F800086B330917307330F8170832B809373077F
:100F900022BB92BB86B330917307330F8170832BD2
:100FA0008093730722BB92BB86B330917307330FD4
:100FB0008170832B8093730722BB92BB86B33091E1
:100FC0007307330F8170832B8093730722BB92BB0F
:100FD00086B330917307330F8170832B809373072F
:100FE00022BB92BB86B390917307990F8170892BB6
:100FF000809373078CE182BB089598E092BB880FC1
:10100000816088BB92BB92BB8CE082BB82BB23E039
:1010100028BB92BB92BB82BB82BB28BB92BB92BB5C
:1010200082BB82BB28BB92BB92BB82BB82BB80E0EF
:1010300098E0909379078093780710927307E1E026
:1010400053E048E03CE016C058BB42BB42BB32BB59
:1010500032BB809178079091790796958795909308
:10106000790780937807209173072F5F2093730788
:101070002C3030F486239723892B31F7E8BBE5CF5A
:101080008CE182BB08958823B1F093B39823A9F42F
:101090002CB53DB52135334CB0F31DBC1CBC909133
:1010A00068009F5F90936800993268F384E58093AD
:1010B000690080E008954599EBCF81E00895482FBD
:1010C00050E00DC023B330E0209530952423352324
:1010D000232B49F42CB53DB52135334C30F4811127
:1010E000F1CF459BF7CF81E008951DBC1CBC9091CA
:1010F00068009F5F90936800993288F384E580933D
:10110000690080E008951092680008C093B39823A6
:1011100049F42CB53DB52135334C50F48111F6CF4F
:101120004599F7CF1DBC1CBC1092680081E0089562
:101130001DBC1CBC909168009F5F90936800993221
:1011400068F384E58093690080E008951092680058
:10115000482F50E00DC023B330E020953095242374
:101160003523232B49F42CB53DB52135334C50F4B0
:101170008111F1CF459BF7CF1DBC1CBC10926800BC
:1011800081E008951DBC1CBC909168009F5F909306
:101190006800993268F384E58093690080E00895DF
:1011A0004091680008C093B3982349F42CB53DB52D
:1011B0002135334C58F58111F6CF4599F7CF809101
:1011C000760790917707BC016F5F7F4F7093770729
:1011D000609376072CB5FC01E759FF4F20839C01F3
:1011E0002E5F3F4F30937707209376075DB5FB0165
:1011F000E759FF4F508303969093770780937607C4
:10120000F901E759FF4F408381E008951DBC1CBCE4
:101210004F5F40936800493270F284E58093690023
:1012200080E0089560916800482F50E00DC023B31E
:1012300030E02095309524233523232B49F42CB519
:101240003DB52135334C58F58111F1CF459BF7CF92
:101250008091760790917707AC014F5F5F4F509375
:101260007707409376072CB5FC01E759FF4F2083A1
:101270009C012E5F3F4F30937707209376077DB513
:10128000FA01E759FF4F7083039690937707809395
:101290007607F901E759FF4F608381E008951DBC8F
:1012A0001CBC6F5F60936800693270F284E58093C4
:1012B000690080E00895CF931DBC1CBC10926800AB
:1012C000E09175074E2F50E04930510570F4C82F5A
:1012D000FA01E65DFF4F0C948B0E809167000E942F
:1012E0004308809167000E945F0884E4809369004E
:1012F000CF910895809167000E945F0880916700F8
:101300000E94430884E480936900CF91089595B3C7
:1013100080916700892B85BB1DBC1CBC209162009D
:1013200030E08CB59DB582179307D8F395B38091C3
:1013300067008095892385BB84E480936900CF9101
:10134000089595B3809167008095892385BB1DBC66
:101350001CBC2091620030E08CB59DB582179307CC
:10136000D8F395B380916700892B85BB84E4809383
:101370006900CF91089510927907109278078C2F09
:101380000E94880780917307809374071DBC1CBC62
:101390002CB53DB524313105D8F38C2F0E94880738
:1013A0008091730790917407981748F490916100A9
:1013B000891728F090916000981708F096CF209137
:1013C0007807309179072F5F3F4F3093790720934B
:1013D0007807283C310598F288CF8FE18ABB1BBA89
:1013E0008AE087BB80EF84BB8CE981BB83E085BB4F
:1013F00088E18AB910BC8CE089B986EA80BD80E4B6
:1014000088B982E08EBD1092770710927607C8E205
:1014100074E4572ECC24C394D12CF2E0EF2EF12C9F
:10142000C601895690404C0189E690E03C016094E9
:101430007094A5E02A2ED9E18091760790917707E4
:101440005F9BFECFFC010196909377078093760710
:101450002CB1E759FF4F2083C89FA001C99F500DB1
:1014600011242091690030E02417350748F71092C5
:1014700068001DBC1CBC2091690050926900D0928C
:101480007707C0927607822F90E0FC013197EA3C03
:10149000F10580F0F3E4F093690083E45D9BFECFF7
:1014A0008CB980916900843449F0109277071092CA
:1014B0007607C2CFED5CFF4F0C948B0ED09279076C
:1014C000C09278078091760790917707029768F32A
:1014D00081E090E05D9BFECFFC01E759FF4F8081EA
:1014E0008CB980917807909179070196909379074C
:1014F00080937807209176073091770782179307BA
:1015000048F3D3CF40916D0050916E0060916B0015
:1015100070916C0080916A000E941F0180916900A7
:10152000BDCFA0906B00B0906C0000916D00109149
:101530006E00209164002A9DC0012B9D900D112406
:101540008930974030F4C8014497853D934008F4B2
:1015500042C381E480936900A1CF00916B00109198
:101560006C000930F7E01F07A0F760916D0086EF6F
:10157000860F8B3570F7B0906A0070E08B2D0E945B
:101580005B0940916D00B8018B2D4A3009F442C3CC
:101590000E9430028091690081CFA0906A00B090D3
:1015A0006B0000916C0010916D0080916400A501AA
:1015B000440F551F849F9001859F300D11242930C1
:1015C000374038F6980124513109253D334008F65B
:1015D000F0927707E092760780936A00B80180E086
:1015E0000E945B09B801C5010E94F804809169005E
:1015F00055CF00916B0010E0102F002780916A00FA
:10160000082B109379070093780730906C001092A4
:101610007407332009F412C38AE6A82E80E0B82E9E
:10162000412C060D171DC4018A0D9B1D9093770751
:1016300080937607C8018A0D9B1D0E949A0EF501C2
:1016400081935F014394409274073410ECCF8091F2
:10165000690024CF80916B0090E0982F882720911B
:101660006A00822B909379078093780760916C00D1
:101670000E94A20E8091690011CF00916A00109122
:101680006B00C801880F991F8930974008F061CF1F
:1016900060916C0086EF860F8B3508F05ACF70E0B2
:1016A00080E00E945B0960916C00C8010E94DF022B
:1016B00080916900F3CE60916B0070916C00809115
:1016C0006A000E94FD0780916900E8CE80916A005F
:1016D0008111B6C280916B008BBB80916900DECE18
:1016E00080916A008111CAC280916B008ABB80918F
:1016F0006900D4CE80916A008093620084E4CECEEB
:1017000080916A008770886183BF80916B008CBF75
:1017100080916900C3CE88E683BDD5BD1DBC1CBCCD
:101720008CB59DB5843C9940D8F315BC1DBC1CBC40
:101730008CB59DB5843F9140D8F380916A00809329
:10174000740710927307D5BD1DBC1CBC8CB59DB52C
:10175000843F9140D8F315BC1DBC1CBC8CB59DB515
:10176000843F9140D8F38091740787FD32C0880F81
:1017700080937407809173078F5F8093730788301D
:1017800010F3D5BD1DBC1CBC8CB59DB5843F9140EC
:10179000D8F315BC1DBC1CBC8CB59DB5843F9140D5
:1017A000D8F3809169007ACE80916A00811137C2A6
:1017B000F0927707E092760789B380936A0084E419
:1017C0006DCE80916A00811165C213BE809169005F
:1017D00065CE1DBC1CBC2CB53DB5243F3140D8F3B3
:1017E000C6CF80916A00882381F38CBF8BE683BFCC
:1017F0008091690053CE80916A00883008F03AC227
:1018000087B988E080BF16B88091690047CE809183
:101810006A00F0E18F9FC0011124836085BB809135
:1018200069003CCE80916A008093660084E436CEE5
:1018300080916A008093610080916B0080936000CA
:1018400084E42CCE80916A008F70809374071DBC55
:101850001CBC0E945F08882309F4F9CE80917407AC
:101860000E948308882309F4F2CE809174070E94B5
:101870005F08882309F4EBCE80916B009FEF980FEF
:1018800090936B00882361F0809174070E94430855
:10189000882331F0809174070E945F088111ECCF9A
:1018A00080916900843509F4F9CD809174070E9414
:1018B000D00880916900F2CD80916A00853008F0EF
:1018C000CDC18093750780916B008295807F809356
:1018D000670084E4E3CD80916A008770886185BDEC
:1018E00080916B0083BD80916900D8CD90916A0092
:1018F000892F82958F70809373079F7090937407E0
:101900000E945F08882309F4A2CE809173070E9489
:101910008308882309F49BCE809174070E945F0896
:101920008111C3CF80916900B9CD90916A00892F50
:1019300082958F70809373079F70909374070E94B5
:101940005F08882309F483CE809173070E9483087F
:10195000882309F47CCE809174070E94120980913B
:1019600069009CCD85B390916A00907F892B85BBDF
:10197000109268001DBC1CBC80916A008F700E9490
:101980001209809169008ACD80916A008B3F08F02E
:10199000E0CD8093630084E481CDAC9A1DBC1CBC77
:1019A000809162009CB59817E8F3AC98109268009B
:1019B0001DBC1CBC8CB59DB50597E0F384E00E946E
:1019C000D008809169006ACD27B888E080BF16B83A
:1019D000E0917607F0917707CF0101969093770712
:1019E0008093760723B388B1E759FF4F807290E068
:1019F0009595879595958795922F9770892B8083DC
:101A0000809169004BCD45E050E06AEF71E08AE6D5
:101A100090E00E94910E809176079091770705964D
:101A200090937707809376078091690037CD8091F6
:101A30006A000E94C106909379078093780780918D
:101A40006A000E94C1062091780730917907820FC1
:101A5000931F909379078093780780916A000E9482
:101A6000C1062091780730917907820F931F9093D8
:101A700079078093780780916A000E94C1062091BF
:101A8000780730917907820F931F969587959695E1
:101A90008795909379078093780720917607309106
:101AA0007707F901E759FF4F80832E5F3F4F30934F
:101AB000770720937607918380916900EFCC80911E
:101AC0006A00833008F045CD8093640084E4E6CC5E
:101AD00095B380916A00807F8095892348CF95B324
:101AE00080916A00807F8095892385BB1092680071
:101AF0001DBC1CBC80916A008F700E94D008809130
:101B00006900CCCC90916A00892F807F8093730705
:101B10009F709093740790916600992309F4C0C058
:101B200095B3892B85BB1DBC1CBC809162009CB504
:101B30009817E8F385B3909173079095892385BB37
:101B4000109268001DBC1CBC8CB59DB50597E0F3D8
:101B500080917407243309F012CFCFCF90916A009F
:101B6000892F82958F70809373079F70909374076D
:101B70000E944308882309F46ACD809173070E946C
:101B8000A608882309F463CD809174070E94430856
:101B90008111E1CE8091690081CC90916A00892FFA
:101BA00082958F70809373079F70909374070E9443
:101BB0004308882309F44BCD809173070E94A6083F
:101BC000811173CE8091690069CC85B390916A00D0
:101BD000907F892B8ACF40906A00B801842D0E94A3
:101BE0005B0980917607909177079C012F5F3F4FAB
:101BF0003093770720937607FC01E759FF4F209138
:101C000064002083A801B501842D0E94E80380911F
:101C1000690044CC0E948401809169003FCC8130EE
:101C200009F464C0823009F458C0833039F4F0926A
:101C30007707E092760780B380936A0084E42ECC25
:101C4000813009F462C0823009F459C08330B1F7A1
:101C500080916B0082BB8091690020CC893008F0B4
:101C600078CC8093750780916B008F7080936700AC
:101C700084E414CC10BE8091690010CC813039F11D
:101C80008230F9F08330D1F680916B0081BB809176
:101C9000690004CC8CBF89E683BF80916900FECBCC
:101CA00095B38095892385BB1DBC1CBC80916200C7
:101CB0009CB59817E8F395B380917307892B85BB82
:101CC0003FCF80916B0084BB80916900E7CB80910E
:101CD0006B0087BB80916900E1CBF0927707E092BF
:101CE000760783B380936A0084E4D8CBF0927707B9
:101CF000E092760786B380936A0084E4CFCB80912C
:101D00006B0085BB80916900C9CB80916B0088BB5B
:101D100080916900C3CBEE0FFF1F0590F491E02D79
:101D20000994FB01DC0102C005900D924150504026
:101D3000D8F70895E199FECF9FBB8EBBE09A992713
:101D40008DB30895262FE199FECF9FBB8EBB2DBB8F
:101D50000FB6F894E29AE19A0FBE01960895F894AE
:021D6000FFCFB3
:061D6200837D0DC80100A5
:00000001FF
